:1000000012C02AC029C028C027C026C025C024C0CD
:1000100023C022C021C020C01FC01EC01DC01CC0E4
:100020001BC01AC019C011241FBECFEDCDBF10E0F8
:10003000A0E6B0E0E4EBF4E003C0C89531960D9281
:10004000A036B107D1F710E0A0E6B0E001C01D92E4
:10005000A036B107E1F730C0D3CFCF93DF93CDB750
:10006000DEB724970FB6F894DEBF0FBECDBF80ED8C
:1000700097E0A0E0B0E089839A83AB83BC83898159
:100080009A81AB81BC810097A105B10561F089819E
:100090009A81AB81BC810197A109B10989839A83B7
:1000A000AB83BC83ECCF24960FB6F894DEBF0FBEB3
:1000B000CDBFDF91CF910895CCEBD0E0DEBFCDBFB7
:1000C00083E080933A0010923B008FE180933700E9
:1000D000109238008CE78093310010923200198220
:1000E00089818830E0F71B821A828A819B8121E016
:1000F0008C3292070CF0DAC189819927880F991FF9
:10010000880F991F8093380080913B008160809315
:100110003B00A3DF9EEF80913B00892380933B004F
:100120008981992701969D838C838C819D819F83F2
:100130008E832E813F8133232CF48E819F810796FD
:100140009F838E838E819F819595879595958795C1
:1001500095958795880F991F880F991F880F991F6C
:100160002C813D81281B390B932F822F880F991FDB
:10017000880F991F8093380080913B0082608093A4
:100180003B006BDF9DEF80913B00892380933B0018
:1001900089819927029699878887888599859B8781
:1001A0008A872A853B8533232CF48A859B8507968D
:1001B0009B878A878A859B85959587959595879551
:1001C00095958795880F991F880F991F880F991FFC
:1001D00028853985281B390B932F822F880F991F6B
:1001E000880F991F80933800809138008160809338
:1001F000380033DF9EEF80913800892380933800E8
:100200008981992703969D878C878C859D859F87FB
:100210008E872E853F8533232CF48E859F85079608
:100220009F878E878E859F859595879595958795D0
:1002300095958795880F991F880F991F880F991F8B
:100240002C853D85281B390B932F822F880F991FF2
:10025000880F991F809338008091380082608093C6
:100260003800FBDE9DEF80913800892380933800B1
:10027000898199270496998B888B888999899B8B8A
:100280008A8B2A893B8933232CF48A899B89079698
:100290009B8B8A8B8A899B89959587959595879560
:1002A00095958795880F991F880F991F880F991F1B
:1002B00028893989281B390B932F822F880F991F82
:1002C000880F991F8093380080913200846080935A
:1002D0003200C3DE9BEF809132008923809332008D
:1002E0008981992705969D8B8C8B8C899D899F8B05
:1002F0008E8B2E893F8933232CF48E899F89079614
:100300009F8B8E8B8E899F899595879595958795DF
:1003100095958795880F991F880F991F880F991FAA
:100320002C893D89281B390B932F822F880F991F09
:10033000880F991F809338008091320088608093E5
:1003400032008BDE97EF8091320089238093320058
:10035000898199270696998F888F888D998D9B8F93
:100360008A8F2A8D3B8D33232CF48A8D9B8D0796A3
:100370009B8F8A8F8A8D9B8D95958795959587956F
:1003800095958795880F991F880F991F880F991F3A
:10039000288D398D281B390B932F822F880F991F99
:1003A000880F991F8093380080913200806180937C
:1003B000320053DE9FEE8091320089238093320019
:1003C0008981992707969D8F8C8F8C8D9D8D9F8F0E
:1003D0008E8F2E8D3F8D33232CF48E8D9F8D07961F
:1003E0009F8F8E8F8E8D9F8D9595879595958795EF
:1003F00095958795880F991F880F991F880F991FCA
:100400002C8D3D8D281B390B932F822F880F991F20
:10041000880F991F8093380080913200806280930A
:1004200032001BDE9FED80913200892380933200E1
:1004300089819927089699A388A388A199A19BA34C
:100440008AA32AA13BA133232CF48AA19BA107965E
:100450009BA38AA38AA19BA195958795959587953E
:1004600095958795880F991F880F991F880F991F59
:1004700028A139A1281B390B932F822F880F991F90
:10048000880F991F80933800809132008064809398
:100490003200E3DD9FEB80913200892380933200AC
:1004A0008A819B8101969B838A831FCE89818F5F7E
:0404B000898316CE58
:00000001FF
